:100000000C9434000C9451000C9451000C94510049
:100010000C9451000C9451000C9451000C9451001C
:100020000C9451000C9451000C9451000C9451000C
:100030000C9451000C9451000C9451000C945100FC
:100040000C9451000C9451000C9451000C945100EC
:100050000C9451000C9451000C9451000C945100DC
:100060000C9451000C94510011241FBECFEFD4E02A
:10007000DEBFCDBF11E0A0E0B1E0E0EEF0E002C0F5
:1000800005900D92A030B107D9F711E0A0E0B1E0E2
:1000900001C01D92A030B107E1F70E945F000C94EF
:1000A0006F000C9400009C0106C080E09FE0019767
:1000B000F1F72150304021153105B9F70895CFEF00
:1000C000D4E0DEBFCDBF3D9A459A88EE93E00E9412
:1000D0005300459884E690E00E945300F5CFFFCF8F
:00000001FF
